:100000000C9489000C94A6000C94A6000C94A600F5
:100010000C94A6000C94A6000C94A6000C94A600C8
:100020000C94A6000C94A6000C94A6000C94A600B8
:100030000C94A6000C94A6000C94A6000C943A090B
:100040000C94A6000C94A6000C94A6000C94A60098
:100050000C94A6000C94A6000C94A6000C94A60088
:100060000C94A6000C94A6000C94A6000C94A60078
:100070000C94A6000C94A6000C94A6000C94A60068
:100080000C94A6000C94A6000C94A60049324320C0
:10009000535441525420434F4E444954494F4E20EB
:1000A0004552524F520049324320534C415645204D
:1000B00041444452455353204552524F5200493215
:1000C000432044415441205458204552524F52003D
:1000D0004932432044415441205258204552524F06
:1000E00052004932432054494D454F55540049323E
:1000F00043204552524F520A0020545743523D2547
:10010000303278205354415455533D253032780ACB
:10011000000011241FBECFEFD0E1DEBFCDBF11E044
:10012000A0E0B1E0E0EFF0E200E00BBF02C007901A
:100130000D92AA34B107D9F711E0AAE4B1E001C0E9
:100140001D92A635B107E1F70C9464090C940000E8
:100150002F923F924F925F926F927F928F929F92D7
:10016000AF92BF92CF92DF92EF92FF920F931F93C5
:10017000CF93DF93CDB7DEB726970FB6F894DEBFE7
:100180000FBECDBF5C016A017B01522E180127FF13
:1001900002C0552405C085E2821714F485E2582E6A
:1001A000D5019896BE83AD8320E030E040E050E07A
:1001B000C701B6010E94B10E882354F4F101808179
:1001C0009181826091838083F7FAF094F7F8F0943C
:1001D000AE014F5F5F4FC701B6010E94110F3B0197
:1001E0004C01E980FA800B811C8120E030E040E086
:1001F00050E0C801B7010E94B10E8823E9F1CD801B
:10020000DE80442428C02DEC3CEC4CEC5DE3C801BE
:10021000B7010E94410FAE014F5F5F4F0E94110F67
:100220002AE939E941E251E40E94410F0E94960E09
:10023000605DD6016E936D014394E980FA800B8175
:100240001C8120E030E040E050E0C801B7010E948E
:10025000B10E882319F0AC14BD04A8F2750106C0D4
:10026000F60181916F01D7018D937D01ED81FE81B2
:10027000CE16DF06A8F329C020E030E040E050E0D1
:10028000C401B3010E94B40E18161CF07501442479
:100290001CC0442403C04A943701480120E030E0E8
:1002A00040E251E4C401B3010E94410F7B018C0183
:1002B00020E030E040E85FE30E94B10E87FDEBCF25
:1002C000E982FA820B831C837501D1014D915C9107
:1002D00053FF13C0BDEF4B1684F0242D332727FDA9
:1002E0003095852D992787FD909501962817390718
:1002F00024F45460F10151834083D1018D919C918C
:1003000092FD08C05394052D112707FD10950A0D85
:100310001B1D0CC0052D112707FD10950A0D1B1D77
:10032000842D992787FD9095080F191F0A151B0525
:10033000D8F4F5014CC020E030E040E251E4C401C3
:10034000B3010E94410FAE014F5F5F4F0E94110F3A
:100350003B014C0169817A818B819C810E94960EC0
:10036000605DD7016D937D010E151F0528F0ED81AD
:10037000FE81EE16FF06F8F28D819E81081719079F
:1003800018F0F50117A224C0D8018C918B5F8C93D3
:10039000F80131E318C020E3D8012C93A016B10670
:1003A00028F48E918D018F5F8C930DC0D8013C9302
:1003B0004394D1018D919C9192FF05C0AE16BF066A
:1003C00008F420833196D8018C918A3324F7108267
:1003D000842D992787FD909526960FB6F894DEBF59
:1003E0000FBECDBFDF91CF911F910F91FF90EF9086
:1003F000DF90CF90BF90AF909F908F907F906F9045
:100400005F904F903F902F9008952F923F924F9280
:100410005F926F927F928F929F92AF92BF92CF9294
:10042000DF92EF92FF920F931F93CF93DF93CDB79D
:10043000DEB7EE970FB6F894DEBF0FBECDBFCC246B
:10044000DD2476013C017EAF6DAF5A011A8219821C
:10045000FC0117821682838181FDF3C38FEF9FEF2A
:1004600016C409811A8100FFD3C3842D80538A30BA
:10047000D0F4F0E34F1631F4552021F403FD02C00F
:10048000116075C18AE0252D2802C0011124542C69
:10049000580E30ED530E57FE02C04FE7542E03FDA9
:1004A000CAC3352CC8C3442D45564CAF433028F041
:1004B000842D8554833008F0FCC0C501049698AFA4
:1004C0008FABF501C080D180E280F38003FD02C0D4
:1004D00036E0532E077B1A83098346015701A70193
:1004E0009601C701B6010E94970A8823C1F08EE4E5
:1004F0008D838B8381E48C839E012A5F3F4F3AAFCB
:1005000029AF3CAD333008F07AC28B81805E8B839B
:100510008C81805E8C838D81805E8D8370C2C701EB
:10052000B6010E94080F892BE9F089E48D838EE4DF
:100530008C8386E48B8320E030E040E050E0C7010C
:10054000B6010E94B10E87FD06C0AE014A5F5F4F43
:100550005AAF49AFD6CF8DE28E83CE0107969AAFC0
:1005600089AFCFCFC80192609A838983E7E44E16A2
:1005700009F449C0E41544F0F5E44F1679F026E497
:10058000421609F042C31DC036E64316D1F047E6D5
:100590004416C9F155E6451609F037C38E010F5FC1
:1005A0001F4F252DB501A401CE010F960E94A80072
:1005B000282E8CEF380E15140CF43A94DE011F9699
:1005C00015C094609A8389838E010F5F1F4F252D7C
:1005D000B501A401CE010F960E94A800282E151483
:1005E0000CF43A94DE011F96121444F4FD010190BC
:1005F0000020E9F73197CE2ECA1A02C0C52CC39449
:10060000BAAFA9AF7DC1552011F0252D01C021E061
:1006100098609A8389838E010F5F1F4FB501A401F3
:10062000CE010F960E94A800282E89819A8192FF00
:100630001EC0822D850D8150282FA82FBB27A7FD16
:10064000B095AC0FBD1F1F9605C08C91119721501E
:10065000803331F4622F27FD23C02215B4F703C382
:10066000C62E562E5218539400C3C92E17C0252DDE
:10067000E52DFF27E7FDF095EC0FFD1F3F9606C027
:1006800080813197292F2150803379F7922F1216CC
:10069000BCF3522EC22E222309F4EFC2592EEDC212
:1006A000E22FFF27E7FDF095EC0FFD1F108A552480
:1006B00099CFC8018870907003FF04C0552011F4D1
:1006C00021E0522EE9E64E1609F493C0E4153CF100
:1006D000F3E54F1609F474C0F415ACF02BE24216A2
:1006E000E1F1241544F030E24316D1F143E244161F
:1006F00009F080C23FC05DE24516C1F18EE24816A6
:1007000009F078C239C093E64916E1F1E4E64E16E5
:1007100009F46FC0F8E54F1609F06CC29FC020E7DE
:10072000421609F496C0241544F03CE6431641F104
:100730004FE6441609F05EC20DC055E7451609F4B0
:100740008FC0E8E74E1609F489C0F3E74F1609F0A9
:1007500051C221C028E02BAF83C000611A830983F6
:1007600089819A8180629A83898365C200681A832D
:10077000098361C20064FBCF08601A83098352C2F7
:100780000460F5CFA5014E5F5F4F58AF4FABF50149
:10079000C0803A9434C1F501C080D180892B41F0EA
:1007A000652D772767FD7095C6010E949C0C18C0C7
:1007B000F60101900020E9F73197EC19EBAF11C079
:1007C000F501C080D180892B41F0652D772767FD29
:1007D0007095C6010E94910C03C0C6010E94880C4E
:1007E0008BAF95012E5F3F4F38AF2FAB3BAD331A28
:1007F00006C102FF0BC0A5014C5F5F4F58AF4FAB66
:10080000F50160817181828193810EC095012E5F17
:100810003F4F38AF2FABF501808191819C01B90129
:10082000882777FD8095982F6B017C0197FF0BC07F
:1008300002601A830983F094E094D094C094C11CA0
:10084000D11CE11CF11C89819A818F7B9A83898359
:1008500027C000641A83098398E7492E30E13BAF33
:1008600029813A8122FF0BC0A5014C5F5F4F58AF31
:100870004FABF50160817181828193810CC0A5012C
:100880004E5F5F4F58AF4FABF50180819181AC0156
:10089000BA01882799276B017C012F7C3A83298331
:1008A00087017601CE0103969AAF89AF9BADA92E41
:1008B000BB24CC24DD24C801B701A60195010E9408
:1008C0000B106A301CF0640D615201C0605DE9AD2F
:1008D000FAAD6193FAAFE9AFC801B701A60195017E
:1008E0000E940B1079018A0121153105410551053E
:1008F00011F7CC24DD247601CE010396C9ACC81AC9
:1009000049815A81CA0182739070892B09F03A9407
:1009100046FF07C0FBADF03111F482E001C081E079
:10092000381A43FF10C0252D332727FD30958C2D15
:1009300099278217930724F0477F5A83498303C07E
:100940005C18351801C03C1840785170452B69F48B
:10095000832D06C0B30180E290E00E94F70C812F46
:10096000182F11501816B4F3312E89819A8181FF06
:1009700004C0B3018DE290E00BC084FF04C0B3015A
:100980008BE290E005C085FF05C0B30180E290E0F6
:100990000E94F70C89819A8186FF0FC0B30180E322
:1009A00090E00E94F70C2BAD203139F4B301842D77
:1009B000992787FD90950E94F70C89819A8190FF75
:1009C0000DC0832D06C0B30180E390E00E94F70CB8
:1009D000812F182F11501816B4F3312E89819A8166
:1009E00083FF0DC0252D06C0B30180E390E00E9477
:1009F000F70C212F122F11501216B4F3512E8981AA
:100A000087FD0DC0832D06C0B30180E290E00E94F7
:100A1000F70C812F182F11501816B4F3312E33E62E
:100A2000431631F4B3018C2D992787FD9095BEC0F4
:100A300043E74416B1F4460156011BAD09C0F50168
:100A400081915F01B301992787FD90950E94F70C72
:100A50001150A8F76401FBADCF0ED11C2FEF2BAFC7
:100A6000B8C033E54316B1F446018601BBAC08C0FB
:100A7000F8018491B30199270E94F70C0F5F1F4F73
:100A8000BA94FFEFBF16A1F764012BADC20ED11CC3
:100A9000FBAF9FC089819A8191FD03C009AD1AAD5A
:100AA00091C092FF1DC01214BCF4A9ACBAAC122DB7
:100AB00009C0F50181915F01B301992787FD9095E8
:100AC0000E94F70C1150A8F729AD3AAD220D311D47
:100AD0003AAF29AF22240FC0B30180E390E009C0F0
:100AE000E9ADFAAD8191FAAFE9AFB301992787FD7E
:100AF00090950E94F70C15142CF4B3018EE290E04F
:100B00000E94F70C89819A8192FD06C017C0B3013B
:100B100080E390E00E94F70C2394822D815087FFA0
:100B20000DC05A94852D8F5F18168CF307C0B30142
:100B3000892F992787FD90950E94F70CE9ADFAADB2
:100B40009191FAAFE9AF992329F05A94852D8F5FDF
:100B500018166CF389819A8192FD3BC0B301842DF4
:100B6000992787FD90950E94F70C2A9427FE07C0CD
:100B7000B3018DE290E00E94F70C219405C0B3010F
:100B80008BE290E00E94F70C6AE070E0822D9927DA
:100B900087FD90950E94F80F6B017C01CB01C096F8
:100BA000B3010E94F70CB301C701C0960E94F70C75
:100BB00010C0F80182918F01B301992787FD9095AC
:100BC0000E94F70CCE0103960817190791F71AAF88
:100BD00009AF898187FF17C0832D06C0B30180E26A
:100BE00090E00E94F70C812F182F11501816B4F3C3
:100BF000312E09C0B301842D992787FD90950E945D
:100C0000F70CB8AEAFAA1A821982AFA8B8AC13C05D
:100C1000F5E24F1649F481E090E09A8389832AE057
:100C20002BAF3324552407C0B301842D992787FDAA
:100C300090950E94F70C4DAD5EAD4F5F5F4F5EAF7C
:100C40004DAFF301838183FF04C0EDADFEAD449051
:100C500003C0EDADFEAD4080442009F002CCF301AD
:100C60008681978114C0C22E5524EC2DFF27E7FD05
:100C7000F095EC0FFD1F108AB2CCEC2DFF27E7FD9D
:100C8000F095EC0FFD1F108AFEEF4F0E92CCEE9602
:100C90000FB6F894DEBF0FBECDBFDF91CF911F918D
:100CA0000F91FF90EF90DF90CF90BF90AF909F900B
:100CB0008F907F906F905F904F903F902F9008950E
:100CC000EF92FF920F931F93CF93DF93CDB7DEB7D1
:100CD00022970FB6F894DEBF0FBECDBF082F162F98
:100CE0007A0161E088E00E94D808882319F08FEF2C
:100CF0009FEF55C021E048E160E0802F0E94780816
:100D0000882319F08EEF9FEF4AC041E068E2812FFF
:100D10000E941B08882319F08DEF9FEF40C061E00F
:100D200080E10E94D808882319F08CEF9FEF37C02C
:100D300021E040E461E0802F0E947808882319F0C8
:100D40008BEF9FEF2CC021E040E561E0CE010196E2
:100D50000E94B607882319F08AEF9FEF20C021E098
:100D600048E560E0CE0102960E94B607882319F09C
:100D700089EF9FEF14C00E948107882319F088EF44
:100D80009FEF0DC089819927982F88272A813327C3
:100D9000822B932BF7019183808380E090E0229651
:100DA0000FB6F894DEBF0FBECDBFDF91CF911F917C
:100DB0000F91FF90EF900895CF93DF93CDB7DEB7FB
:100DC00022970FB6F894DEBF0FBECDBFAE014F5FC6
:100DD0005F4F62E080E60E94600688231CF48FEF7C
:100DE0009FEF02C089819A8122960FB6F894DEBFE8
:100DF0000FBECDBFDF91CF910895EF92FF920F9379
:100E00001F93CF93DF93CDB7DEB721970FB6F8943A
:100E1000DEBF0FBECDBF082F162F7A0161E088E03C
:100E20000E94D808882319F08FEF9FEF41C021E07E
:100E300048E160E0802F0E947808882319F08EEF47
:100E40009FEF36C041E068E2812F0E941B08882393
:100E500019F08DEF9FEF2CC061E080E10E94D8086F
:100E6000882319F08CEF9FEF23C021E040E461E07C
:100E7000802F0E947808882319F08BEF9FEF18C00D
:100E800021E048E560E0CE0101960E94B607882384
:100E900019F08AEF9FEF0CC00E948107882319F098
:100EA00089EF9FEF05C08981F701808380E090E0A2
:100EB00021960FB6F894DEBF0FBECDBFDF91CF9164
:100EC0001F910F91FF90EF900895CF93DF93CDB7CF
:100ED000DEB721970FB6F894DEBF0FBECDBFAE01CF
:100EE0004F5F5F4F61E080E60E94FD068981992790
:100EF00021960FB6F894DEBF0FBECDBFDF91CF9124
:100F0000089584E980937400E4E7F0E0808184FD33
:100F1000FDCF80E090E00895CF92DF92EF92FF92B4
:100F20000F931F936C01E62E042F0E948107DF921E
:100F3000CF920E94440D11271F930F93FF24FF921D
:100F4000EF9289EF90E09F938F930E94440D8DB7AD
:100F50009EB708960FB6F8949EBF0FBE8DBF1F9127
:100F60000F91FF90EF90DF90CF900895EF92FF9256
:100F70000F931F93FC01342F522F10924B011092AC
:100F80004A01662321F084EC8093740003C084E856
:100F9000809374008091740088233CF080914A0112
:100FA00090914B01885E9340A8F380914A01909103
:100FB0004B01885E9340E0F05523B1F10F2EF1E72D
:100FC000EF2EFF24F02DF701408104E710E0F80137
:100FD000608180ED90E00E948C07F7014081F8016C
:100FE000608182EE90E00E948C078FEF9FEF1EC021
:100FF00040917100842F9927887F9070232F332789
:101000008217930759F0552379F06091740080EDB1
:1010100090E00E948C078FEF9FEF08C080917300D3
:10102000808380E090E002C08FEF9FEF1F910F91CF
:10103000FF90EF900895EF92FF920F931F93542F1C
:1010400010924B0110924A018093730084E88093C0
:101050007400E4E7F0E0808188233CF080914A014D
:1010600090914B01885E9340B0F380914A0190913A
:101070004B01885E9340E0F0552399F10F2EF1E784
:10108000EF2EFF24F02DF701408104E710E0F80176
:1010900060818EEB90E00E948C07F7014081F8019F
:1010A000608182EE90E00E948C078FEF9FEF1BC063
:1010B00040917100842F9927887F9070262F3327C5
:1010C0008217930719F480E090E00DC0552349F092
:1010D000609174008EEB90E00E948C078FEF9FEF81
:1010E00002C08FEF9FEF1F910F91FF90EF90089537
:1010F000EF92FF920F931F93342F522F10924B01B8
:1011000010924A01880F862B8093730084E88093A5
:101110007400E4E7F0E0808188233CF080914A018C
:1011200090914B01885E9340B0F380914A01909179
:101130004B01885E9340E0F0552399F10F2EF1E7C3
:10114000EF2EFF24F02DF701408104E710E0F801B5
:10115000608186EA90E00E948C07F7014081F801E7
:10116000608182EE90E00E948C078FEF9FEF1BC0A2
:1011700040917100842F9927887F9070232F332707
:101180008217930719F480E090E00DC0552349F0D1
:101190006091740086EA90E00E948C078FEF9FEFC9
:1011A00002C08FEF9FEF1F910F91FF90EF90089576
:1011B000EF92FF920F931F93282F10924B011092E2
:1011C0004A0184EA80937400E4E7F0E08081882398
:1011D0003CF080914A0190914B01885E9340B0F3BE
:1011E00080914A0190914B01885E9340E0F0662324
:1011F00061F10F2EF1E7EF2EFF24F02DF701408172
:1012000004E710E0F80160818CE890E00E948C0710
:10121000F7014081F801608182EE90E00E948C0726
:101220008FEF9FEF14C040917100421719F480E0D6
:1012300090E00DC0662349F0609174008CE890E066
:101240000E948C078FEF9FEF02C08FEF9FEF1F91DF
:101250000F91FF90EF9008959C0112BE10924B01E8
:1012600010924A0180914A0190914B018217930795
:10127000C9F708951F920F920FB60F9211248F9302
:101280009F9380914A0190914B01019690934B015D
:1012900080934A019F918F910F900FBE0F901F90E6
:1012A000189513BE86B7836086BF87B7836087BFF4
:1012B0008DE083BF12BE8DE781BF08955D9BFECF99
:1012C0008CB980E090E00895CFEFD0E1DEBFCDBFD4
:1012D0000E9451091092900087E689B988E08AB986
:1012E000789460E070E08EE599E00E94A70CE1E759
:1012F000F0E080818C7F80838CE180937000E4E754
:10130000F0E080818460808388EE93E00E942C0965
:101310000E94DC06992304F19C01B901882777FD1E
:101320008095982F0E94CE0F20E030E040E251E4FB
:101330000E94DD099F938F937F936F9380E091E0EC
:101340009F938F930E94240D8DB79EB706960FB67C
:10135000F8949EBF0FBE8DBF0E946507182F682F9F
:10136000772767FD7095872F972F0E94CE0F112347
:1013700034F420E030E040E853E40E948A0F20E09B
:1013800030E044EB5FE30E94410F9F938F937F9384
:101390006F938EE191E09F938F930E94240D8AE0DA
:1013A00090E00E94730D2DB73EB72A5F3F4F0FB6F6
:1013B000F8943EBF0FBE2DBFA7CFA8E1B0E0E3EE8B
:1013C000F9E00C94471069837A838B839C832D8387
:1013D0003E834F835887B9E08B2E912C8C0E9D1E37
:1013E000B401CE0101960E94E90B8E010F5E1F4FE2
:1013F000B801CE0105960E94E90B2985223008F438
:101400006AC03989323008F468C08A859A89892788
:101410008A87243009F463C0223009F460C0343074
:1014200041F41D861E861F86188A1C861B86B40101
:1014300077C0323009F458C06B857C858B899C89D4
:10144000681B790B7C876B872D853E854F85588976
:10145000ED88FE880F89188D2E153F05400751072E
:1014600040F4220F331F441F551F615070407C878A
:101470006B8780E090E0A0E0B0E4AA24BB24650183
:1014800060E070E02E153F054007510740F0A82AA4
:10149000B92ACA2ADB2A2E193F09400B510BB695EF
:1014A000A79597958795220F331F441F551F6F5F90
:1014B0007F4F6F31710531F7D601C5018F7790707D
:1014C000A070B07080349105A105B10589F0AD869A
:1014D000BE86CF86D88AB40123C0B80121C0321796
:1014E000D1F76CE371E01CC084E08987B40118C0B7
:1014F000A7FCEDCF211531054105510541F380E4ED
:1015000090E0A0E0B0E0A80EB91ECA1EDB1E80E885
:101510009FEFAFEFBFEFA822B922CA22DB22D7CFBD
:10152000CB010E94C70AECE068960C946310A8E116
:10153000B0E0EDE9FAE00C94511069837A838B8373
:101540009C832D833E834F835887BE01675F7F4F07
:10155000CE0101960E94E90BBE016F5E7F4FCE0166
:1015600005960E94E90B8985823018F481E090E0AD
:101570000AC020E030E08989823010F0C90103C040
:1015800021E030E0C901E2E068960C946D104F92C2
:101590005F926F927F928F929F92AF92BF92DF92F3
:1015A000EF92FF920F931F9320E030E040E050E075
:1015B000FC01E480F58006811781D1808081823032
:1015C00038F4D801C701A061AF77B0706FEFD9C010
:1015D000843009F46EC0823009F471C0E114F10462
:1015E0000105110509F46BC0828193816FEF823888
:1015F00096070CF06AC062E87FEF681B790B6A31CE
:1016000071050CF080C047015801062E04C0B69445
:10161000A794979487940A94D2F7442455243201CE
:1016200081E090E0A0E0B0E004C0880F991FAA1FFD
:10163000BB1F6A95D2F70197A109B109E822F922E7
:101640000A231B23E114F1040105110529F061E0CF
:10165000462E512C612C712C85017401E428F5284B
:1016600006291729D801C7018F779070A070B07034
:1016700080349105A105B10509F457C0D801C7010F
:10168000CF96A11DB11D60E070E08030E0E09E07C4
:10169000E0E0AE07E0E4BE0710F061E070E027E0B4
:1016A000B695A795979587952A95D1F7AF77B0709E
:1016B00068C080E090E0A0E0B0E06FEF62C080E042
:1016C00090E0A0E0B0E060E05CC0803891058CF76D
:1016D000BC0161587F4FD801C7018F779070A0700F
:1016E000B07080349105A105B105A1F08FE390E0C1
:1016F000A0E0B0E0E80EF91E0A1F1B1F17FD28C06E
:10170000D801C701CCCF60E070E080E090E0A0E0BD
:10171000B0E0CCCFE7FEF2CF80E490E0A0E0B0E014
:10172000E80EF91E0A1F1B1FE9CFE7FC18C080E076
:1017300090E060E0E61660E0F60660E0060760E430
:10174000160710F081E090E0BC01D801C701A7CFD7
:1017500016950795F794E7946F5F7F4FD1CFD80127
:10176000C701805C9F4FAF4FBF4F60E070E080309B
:10177000E0E09E07E0E0AE07E0E4BE0708F48FCFAC
:101780008CCF282F392F9A2F9F77842F8078892B01
:10179000962F9795992797958F77482F492B669580
:1017A000852F8078862BD794DD24D7948F77582F78
:1017B0005D29CA01B9011F910F91FF90EF90DF9051
:1017C000BF90AF909F908F907F906F905F904F9061
:1017D0000895FC01DB01208131819281492F4F77EF
:1017E00050E0991F9927991F8381682F660F692BF5
:1017F000881F8827881FFD018183662309F049C05F
:10180000211531054105510509F470C082E89FEFAB
:10181000FD0193838283220F331F441F551F220F24
:10182000331F441F551F220F331F441F551F220F04
:10183000331F441F551F220F331F441F551F220FF4
:10184000331F441F551F220F331F441F551F83E0B2
:101850008C932030F0E03F07F0E04F07F0E45F07A3
:1018600090F482E89FEF220F331F441F551F01970A
:10187000203060E0360760E0460760E4560798F3E2
:10188000FD0193838283FD0124833583468357833F
:1018900008956F3F71F1862F99278F579040FD0172
:1018A0009383828383E08C93220F331F441F551F41
:1018B000220F331F441F551F220F331F441F551F74
:1018C000220F331F441F551F220F331F441F551F64
:1018D000220F331F441F551F220F331F441F551F54
:1018E00050642483358346835783089582E08C9324
:1018F0000895211531054105510519F484E08C93B3
:10190000089544FD02C01C92BECF81E08C93BBCFF2
:10191000FC0105900020E9F7809590958E0F9F1FA0
:101920000895FC010590615070400110D8F7809532
:1019300090958E0F9F1F0895FC016150704001909B
:101940000110D8F7809590958E0F9F1F0895EF9204
:10195000FF920F931F93CF93DF938C017B01892B11
:1019600011F4672BD1F16EE070E081E090E00E940D
:101970007A0DFC01009789F1DC0180E88383E11492
:10198000F10471F0F386E28681E8838380914C0153
:1019900090914D01892B21F4F0934D01E0934C017E
:1019A00001151105E1F0118700878381826083832F
:1019B00080914E0190914F01892B89F4F0934F0152
:1019C000E0934E018091500190915101892B39F49F
:1019D000F0935101E093500102C0A0E0B0E0CD01CE
:1019E000DF91CF911F910F91FF90EF9008950F938A
:1019F0001F93CF93DF938C01EB018B81992781FF9C
:101A00001BC082FF0DC02E813F818C819D812817D4
:101A1000390764F4E881F9810193F983E88306C00A
:101A2000E885F985802F0995892B31F48E819F8176
:101A300001969F838E8302C00FEF1FEFC801DF91D5
:101A4000CF911F910F910895CF93DF93CDB7DEB75C
:101A500022970FB6F894DEBF0FBECDBFFE013796BA
:101A600061917191FA83E983AF0180914E01909168
:101A70004F010E94050222960FB6F894DEBF0FBEFA
:101A8000CDBFDF91CF910895CF93DF93CDB7DEB770
:101A900022970FB6F894DEBF0FBECDBFFE0137967A
:101AA00061917191FA83E983E0914E01F0914F01C8
:101AB00083818860838349815A8180914E0190910E
:101AC0004F010E940502E0914E01F0914F012381E8
:101AD000277F238322960FB6F894DEBF0FBECDBFBB
:101AE000DF91CF91089560914E0170914F010E9456
:101AF000F70C08950F931F93CF93DF93869F800178
:101B0000879F100D969F100D1124C8010E94960DFD
:101B1000EC01009729F0A80160E070E00E948F0EB0
:101B2000CE01DF91CF911F910F910895CF93DF9355
:101B3000AC01029710F442E050E0A0915401B09142
:101B40005501FD01C0E0D0E020E030E020C0808100
:101B500091818417950769F482819381209719F008
:101B60009B838A8304C09093550180935401CF01D5
:101B700032C04817590738F42115310519F082177A
:101B8000930708F49C01EF010280F381E02D309768
:101B9000F1F62115310589F1C901841B950B0497D4
:101BA00008F4A901E0E0F0E026C08D919C91119726
:101BB00082179307E9F44817590779F4ED018A81F0
:101BC0009B81309719F09383828304C090935501D1
:101BD00080935401CD01029649C0841B950BFD01F1
:101BE000E80FF91F4193519302978D939C933AC04C
:101BF000FD01A281B3811097C1F6809152019091AD
:101C00005301892B41F480914601909147019093B3
:101C100053018093520120914801309149012115CF
:101C2000310541F42DB73EB78091440190914501B3
:101C3000281B390BE0915201F09153012E1B3F0BF1
:101C40002417350788F0CA0102962817390760F073
:101C5000CF01840F951F02969093530180935201F8
:101C600041935193CF0102C080E090E0DF91CF918A
:101C70000895CF93DF93009709F44EC0EC012297AB
:101C80001B821A82A0915401B0915501109711F155
:101C900040E050E001C0DC01AC17BD0700F1BB83A0
:101CA000AA83FE0121913191E20FF31FEA17FB078E
:101CB00071F42E5F3F4F8D919C911197820F931F6E
:101CC00099838883FD01828193819B838A83411557
:101CD000510559F4D0935501C09354011DC0FD0125
:101CE00082819381AD010097B1F6FA01D383C2835B
:101CF00021913191E20FF31FEC17FD0769F42E5F7C
:101D00003F4F88819981820F931FFA0191838083CD
:101D10008A819B8193838283DF91CF910895DC0137
:101D200001C06D9341505040E0F7089597FB47D0B4
:101D30009F3738F0FEE9F91B982F872F762F6B2FEE
:101D400005C05AC09695879577956795F150D0F75D
:101D50003EF490958095709561957F4F8F4F9F4F82
:101D600008950ED05EF004C00BD026F001C008D05C
:101D700019F020F48FEF089580E0089581E0089530
:101D800097FB092E052600F8689410D0E89407FC0C
:101D900007C0621773078407950721F008F40094C1
:101DA000079498940895052E092607FA440F551FA5
:101DB0005F3F79F0AA27A51708F051E04795880FF3
:101DC000991F9F3F31F0BB27B91708F091E0879525
:101DD00008959F919F91112408C197FB880F991F27
:101DE0009F3F31F0BB27B91708F091E08795089520
:101DF0009F919F911124F9C06627772788279927FB
:101E000008959F3F59F4803C49F481E09927089553
:101E100090688923872386238395B9F38827992798
:101E20000895DBDFCF93DF93D52FC42F55274427A9
:101E3000332722279923D9F09F37C8F0F92FBDD037
:101E4000592F482F372F262FF63968F46FDFA6D089
:101E5000C030CD0721F06993799389939993905875
:101E6000DF91CF9157C09927882777276627C03001
:101E7000CD0721F02993399349935993DF91CF915D
:101E80009CC091DF01D099C0992339F0552329F0E6
:101E90009F575F57950F13F49AF1B1CF91589F3F19
:101EA000E1F3629FA12D0F92BB27639FA00DB11D8F
:101EB000EE27729FA00DB11DEE1FAF93AA27649F5E
:101EC000B00DE11D739FB00DE11DAA1F6627829F13
:101ED000B00DE11DA61F5527749FE00DA11D551FD4
:101EE000839FE00DA11D561F849FA00D511D852FBE
:101EF0007A2F6E2F1F900F9088231AF4939539F440
:101F000074C0000C111CBB1F661F771F881F01289F
:101F100008955058192E47DF01D04FC0BA176207F5
:101F2000730784079507B1F188F40EF410940B2E13
:101F3000BA2FA02D062E622F202D072E732F302DA5
:101F4000082E842F402D092E952F502DFF27552325
:101F5000B9F0591B49F0573E98F0469537952795AB
:101F6000A795F0405395C9F776F0BA0F621F731F1B
:101F7000841F30F4879577956795B795F0409395D2
:101F800017FA0F2E0895BF1BBB27BA0B620B730BFA
:101F9000840BF6CFDEF633CFE89403C097FB0EF444
:101FA000D8DEB62F672F782F892F9EE9002405C031
:101FB0009A95BB0F661F771F881F11249923A1F0E4
:101FC0008823B2F79F3F59F0BB0F48F421F400205B
:101FD00011F460FF04C06F5F7F4F8F4F9F4F881FCA
:101FE0009795879597F9089507CF9FEF80EC08950F
:101FF00097FB092E07260AD077FD04D02ED006D0F5
:1020000000201AF4709561957F4F0895F6F790952A
:1020100081959F4F0895A1E21A2EAA1BBB1BFD01BB
:102020000DC0AA1FBB1FEE1FFF1FA217B307E407B7
:10203000F50720F0A21BB30BE40BF50B661F771F0F
:10204000881F991F1A9469F76095709580959095EF
:102050009B01AC01BD01CF010895AA1BBB1B51E13F
:1020600007C0AA1FBB1FA617B70710F0A61BB70B08
:10207000881F991F5A95A9F780959095BC01CD01AD
:1020800008952F923F924F925F926F927F928F921C
:102090009F92AF92BF92CF92DF92EF92FF920F93F7
:1020A0001F93CF93DF93CDB7DEB7CA1BDB0B0FB601
:1020B000F894DEBF0FBECDBF09942A8839884888BE
:1020C0005F846E847D848C849B84AA84B984C88454
:1020D000DF80EE80FD800C811B81AA81B981CE0F4B
:1020E000D11D0FB6F894DEBF0FBECDBFED01089530
:1020F00062656172696E672028313629203D20258E
:10210000302E316620646567726565730A0062650A
:102110006172696E672028382920203D2025302EE5
:10212000316620646567726565730A00000000000F
:0A213000000000002000560100002E
:00000001FF
